:040000006F00F00895
:100004000000000000000000EE050000F005000004
:10001400000000008C080000000000000000000048
:100024008C0800008C0800000000000000000000A4
:100034007A1500000000000000020000000000002B
:100044008C0800008C0800008C0800008C0800005C
:100054008C0800008C0800008C0800008C0800004C
:100064008C0800008C0800008C0800008C0800003C
:100074008C0800008C0800008C0800008C0800002C
:100084008C0800008C0800008C0800008C0800001C
:100094008C0800008C0800008C0800008C0800000C
:1000A4008C0800008C0800008C0800008C080000FC
:1000B4008C0800008C0800008C0800008C080000EC
:1000C4008C0800008C0800008C0800008C080000DC
:1000D4008C0800008C080000243900006E390000F0
:1000E4008C0800008C0800008C0800008C080000BC
:1000F4008C0800008C0800008C0800008C080000AC
:10010400000000008C0800008C0800008C0800002F
:100114008C080000B83900008C0800008C0800002E
:100124008C0800008C0800008C0800008C0800007B
:100134008C0800008C0800008C0800008C0800006B
:100144008C0800008C0800008C0800008C0800005B
:100154008C0800008C0800008C080000023A0000A3
:100164004C3A0000963A00008C0800008C0800000D
:100174008C0800008C0800008C0800008C0800002B
:100184008C0800008C0800008C0800008C0800001B
:100194008C0800008C0800008C0800008C0800000B
:1001A400000000000000000000000000000000004B
:0C01B4000000000000000000000000003F
:10020000130181F806C216C41AC61EC822CA26CC1B
:100210002ACE2ED032D236D43AD63ED842DA46DC76
:100220004ADECEC0D2C2D6C4DAC6DEC8E2CAE6CC46
:10023000EACEEED0F2D2F6D4FAD6FED8F3220030CF
:1002400096DA9702002083A2A20023A02200F325C1
:1002500010342EC09305000273A0458003A1C18114
:10026000EF20A04517030020032383FE0321030092
:10027000824273901234D652739002309240A2425E
:100280003243C2435244E244724582551256A2564A
:100290003257C2575258E25872598649164AA64AEE
:1002A000364BC64B564CE64C764D865D165EA65ECA
:1002B000365FC65F13018107730020301300000012
:1002C00013000000130000001300000013000000E2
:1002D00013000000130000001300000013000000D2
:1002E00013000000130000001300000013000000C2
:1002F00013000000130000001300000013000000B2
:1003000083A2C181938202E073900234170100201E
:10031000032101F4024182403243C2435244E24489
:10032000724582551256A2563257C2575258E25859
:1003300072598649164AA64A364BC64B564CE64C6D
:10034000764D865D165EA65E365FC65FD652A1020A
:1003500073900230A24213018107828013000000D3
:100360001300000013000000130000001300000041
:100370001300000013000000130000001300000031
:100380001300000013000000130000001300000021
:100390001300000013000000130000001300000011
:1003A0001300000013000000130000001300000001
:1003B00013000000130000001300000013000000F1
:1003C00013000000130000001300000013000000E1
:1003D00013000000130000001300000013000000D1
:1003E00013000000130000001300000013000000C1
:1003F00013000000130000001300000013000000B1
:10040000F322003093F272FF130380781203B3E2F9
:100410006200711523205500130585FA10C12115BE
:10042000232005009302000063870200711523203A
:100430000500FD12D5BF71150CC1828000000000BF
:1004400000000000000000000000000000000000AC
:10045000000000000000000000000000000000009C
:10046000000000000000000000000000000000008C
:10047000000000000000000000000000000000007C
:10048000000000000000000000000000000000006C
:10049000000000000000000000000000000000005C
:1004A000000000000000000000000000000000004C
:1004B000000000000000000000000000000000003C
:1004C000000000000000000000000000000000002C
:1004D000000000000000000000000000000000001C
:1004E000000000000000397101436EC619A0397187
:1004F00041536AC866CA62CC5ECE19A039710153F5
:100500005AD056D252D44ED64AD826DA22DC06DE4B
:1005100033016140828241114AC026C222C406C60C
:100520008282B24D4101024D924C224CB24B4101AC
:10053000024B924A224AB249410102499244224462
:10054000B240410182803D432A876373C30293779F
:10055000F700BDEFADE5937606FF3D8ABA960CC372
:100560004CC30CC74CC74107E36BD7FE11E2828036
:10057000B306C3408A069702000096966780A600DD
:100580002307B700A306B7002306B700A305B700EB
:100590002305B700A304B7002304B700A303B700E3
:1005A0002303B700A302B7002302B700A301B700DB
:1005B0002301B700A300B7002300B700828093F5A2
:1005C000F50F93968500D58D93960501D58D61B76E
:1005D000939627009702000096968682E78086FA17
:1005E0009680C1171D8F3E96E374C3F8A5B701A08E
:1005F000B707EFBE37E700E0938707083CC701A0C5
:10060000EFF27FF10945EF00100A912AEF20F00682
:10061000716513050520EF207009B707002083A539
:100620000720376500001305C567EF40D05FCD2375
:10063000AA85376500001305C568EF40D05EB76531
:100640000000376500009385C5691305456AEF40D2
:10065000905DEF400007376400001305446CEF40E5
:10066000D06DE5BFB71702409843B706FFF04111C0
:100670001367170098C3D84337060200758FD8C395
:100680009843B706F7FEFD16758F98C39843B706D3
:10069000FCFFFD16758F98C3D843B70601FFFD1602
:1006A000758FD8C39843B70600ECFD16758F98C3B5
:1006B0003707FF0098C723A6070202C402C6984363
:1006C000C166558F98C3B716024005679C42F18FEB
:1006D0003EC6A24785073EC4B24781E7A247E397DB
:1006E000E7FEB71702409C431397E70063570706DE
:1006F00085473EC632478547631FF704B717024058
:10070000D843B706C1FFFD16D8C3D843D8C3D843D2
:1007100013670740D8C3D843758FD8C3D843B706EB
:100720001100558FD8C39843B7060001558F98C361
:10073000984393166700E3DD06FED843B7160240E0
:10074000719BD8C3D84313672700D8C32147DC4225
:10075000B18BE39EE7FE4101828002C661BFB716FE
:100760000240D842B70700201146318B93870720FB
:100770006305C70021466308C70237177A001307CD
:10078000072098C337170240584311839376F70028
:100790003707002013070700369714239843335771
:1007A000D70098C38280D842D442416649833D8BAA
:1007B000F18E1306270015CF3D47630FE602414730
:1007C000630FE602454781456313E6004146A1E217
:1007D0003747024003270780418B0DC737177A0040
:1007E000130707203306C70290C3C9DD984305836A
:1007F00049BF81454946E1BF85453546C9BF814569
:100800003D46F1B737173D0013070790E1BF371595
:10081000024058559316F700585563DF06041183BC
:100820003D8B9306170037177A00130707203357BD
:10083000D70298C35455A182BD8A8DE295463307ED
:10084000D702058398C337170240585794433D8B0E
:10085000050733D7E60298C3984369B70545639403
:10086000A600E546E9BF3D456396A600D14633871D
:10087000E602C9BF8906E5BF3D8B9306170037170F
:100880007A00130707203357D702F1B701A0970169
:10089000002093812117177100201301A17617659D
:1008A00000001305250A97F5FF1F9385A57513868C
:1008B000818263FAC5008322050023A0550011053B
:1008C0009105E3EAC5FE17050020130525969765F7
:1008D00000209385A5506377B500232005001105FE
:1008E000E36DB5FEFD42739002BCFD427390428001
:1008F000B7820000938202807390023097F2FFFF6C
:100900009382827093E2320073905230EFF09FD561
:1009100097020000938202CF73901234730020304C
:10092000EFF27FBFB727014093870740631BF500B5
:100930008545130500207D278145130500205D278F
:10094000EDBEB737014093870780E31BF5FE854571
:1009500013050040412F814513050040CDB75C4190
:100960003707F1E01307F7EF944D7D8F9C41D58F4A
:10097000D44DD58FD441A206D58FD98F5CC11C45EB
:1009800037F7F1FF1307D77FD4457D8F9C49D58F6B
:1009900094458606D58FD98F1CC55C55370710FF47
:1009A0007D177D8FDC29FD1793F7F70FD207D98FBD
:1009B0005CD582801C4589C593E717001CC58280E1
:1009C000F99BEDBF1C4589C593E707101CC58280C4
:1009D00093F7F7EFE5BF1C4593E787001CC58280BE
:1009E00008450D81058982801C4593E747001CC599
:1009F000828008450981058982801C4591C5370799
:100A00005000D98F1CC582803707B0FF7D17F98F42
:100A1000D5BFA54763F7B7048D47138765FF330735
:100A2000F7020328C5009D47B397E70093C7F7FF78
:100A3000B3F70701B396E600DD8E54C5994763E32B
:100A4000C70495477D163306F6025859FD47B397FC
:100A5000C70093C7F7FFF98F3396C5005D8E50D955
:100A600082800D473387E502032805019D47B39730
:100A7000E70093C7F7FFB3F70701B396E600DD8EF3
:100A800014C96DBFB14763E2C702954765163306C7
:100A9000F6021859FD47B397C70093C7F7FFF98FC0
:100AA0003396C5005D8E10D9828095474D1633066A
:100AB000F6025855FD47B397C70093C7F7FFF98F64
:100AC000B395C500DD8D4CD582805C4191C537075B
:100AD0000004D98F5CC18280370700FC7D17F98F35
:100AE000D5BFEFF25FA301112A8423040100A544BE
:100AF0001C8463F8F40423040100A54621461C84E9
:100B000063FCF606231501002304010095461C84AE
:100B100063FEF60C38853C8599460D46B3F7D7023F
:100B2000056513050580B3D7C7023357D702BA97B7
:100B3000C207C1837C853C8505611D8D42054185C9
:100B4000EDBA1C4493E787001CC42285513D75FD16
:100B50001C4493E747001CC42285613D75FD784421
:100B60001C8414108607B6972396E7FE1C8485071D
:100B700093F7F70F5C84ADBFA30401009C846378F6
:100B8000F6001C84850793F7F70F5C848DBF98846B
:100B90009C840C100607850786072E97AE9703578F
:100BA000C7FE83D7C7FE63FDE7029C848607AE9726
:100BB00083D7C7FE7C859C84988485078607AE977B
:100BC00083D5C7FE931717001810BA972396B7FE60
:100BD0009C8438850C1085078607AE972396E7FE20
:100BE0009C84850793F7F70FDC8449BF1C841010A1
:100BF000388589078607B29783D7C7FEBA97C20799
:100C0000C1837C851C84850793F7F70F5C8401B74B
:100C1000B7F7FF1F03A5477082801C414167791712
:100C2000F98F1CC123200500232205002324050081
:100C3000B707024023260500138787006317E500E6
:100C4000D8431367F700D8C382801387C7016316A0
:100C5000E500D8431367070FFDB713870703631831
:100C6000E500D8438566938606F0558FE9BF138764
:100C700047046315E500D843BD66C5BF13878705E4
:100C80006316E500D843B7060F00C5B71387C7063C
:100C90006316E500D843B706F000C1BF1387070805
:100CA0006316E500D843B706000FC1B71387874026
:100CB0006319E50003A747401367F70023A2E74045
:100CC00082801387C7416317E50003A74740136776
:100CD000070FEDB793870743631BF500B707024083
:100CE00003A747408566938606F0558FC1BFB707B7
:100CF0000240138747446316E50003A74740BD66DB
:100D0000EDB7138787456317E50003A74740B7068C
:100D10000F00E1BF1387C7466317E50003A74740ED
:100D2000B706F000D9B7138707486317E50003A794
:100D30004740B706000F55BF138707496319E50001
:100D400003A7474D1367F70023AAE74C8280138758
:100D5000074A6317E50003A7474D1367070FEDB771
:100D60001387074B6319E50003A7474D85669386F4
:100D700006F0558FD1BF1387074CE319E5FC03A795
:100D8000474DBD66FDB71C4161773D0794517D8F8E
:100D90009C45D58F9449D58FD449D58F944DD58F07
:100DA000D44DD58FD451D58F9455D58FD98F1CC1A3
:100DB000DC455CC19C411CC5DC415CC582801C419A
:100DC00089C593E717001CC1828041677917F98FA5
:100DD000DDBF9C4513F7070113F8F70001C7D841A1
:100DE0003368E8008E2113F7F50F39C318418146A7
:100DF000854E3D4F930F800293028004214E33961F
:100E0000DE00B3F8C5006311160393982600331370
:100E10001F011343F3FF3377E300B318180133E7DF
:100E2000E800639FF70550C98506E39AC6FD18C11F
:100E30001307F00F6375B70454412146854E3D4FAB
:100E4000930F800293028004414EB398CE0033F793
:100E500015016392E8021317260001173313EF0000
:100E60001343F3FFB376D3003317E800D98E639DA5
:100E7000F701232A15010506E319C6FD54C1828036
:100E8000E39457FA10C94DB7E39757FE232815018D
:100E9000DDB748456D8D3335A000828019C20CC97D
:100EA00082804CC98280B707002023A4A7228280B9
:100EB000B707002003A78722894710216311F70293
:100EC00014318D4763EDD7003C219A0637E700E0E7
:100ED0009607D58F93F7F70F32972300F7405441C9
:100EE0000547935756003317C70089CA93870704ED
:100EF0008A07B7E600E0B69798C382809387070613
:100F0000C5BFB7160240DC4251777D17F98F5D8D62
:100F1000C8C28280371702405C439146B18B63851B
:100F2000D700A1466382D706B7177A0093870720B8
:100F30001CC1371602405C42370700201307070127
:100F40009183BD8BBA9794231C41B3D7D7005CC162
:100F50005442A1829D8ABA969422B3D6D70014C572
:100F60005442AD829D8A36971823B3D7E7005CC5FB
:100F70005842398393763700138741803697182378
:100F8000B3D7E7021CC982805C435843C166C9835A
:100F9000758FB7F6FF1F83A6C670BD8B89071396A2
:100FA000160163480600C54601466392D702C94749
:100FB00039A88946638FD702BD46638ED702C146E2
:100FC000638ED702C54601466393D700C1471DEF24
:100FD0003747024003270780418B05C737177A0040
:100FE00013070720B307F7021CC121D61C418583D4
:100FF00081B701466DBF0546B547D1BF0146BD4724
:10100000F9B737173D0013070790E9BFB71502403E
:10101000D8559316F700D85563DF060411833D8B2E
:101020009306170037177A00130707203357D702A4
:1010300018C1D455A182BD8A8DE295463307D702E7
:10104000058318C137170240585714413D8B0507D7
:1010500033D7E60218C1184171B785456394B600CD
:10106000E546E9BFBD456396B600D1463387E60243
:10107000C9BF8906E5BF3D8B9306170037177A0075
:10108000130707203357D702F1B799C53717024026
:101090005C4B5D8D48CB8280B7170240D84B13451F
:1010A000F5FF798DC8CB828099C5371702401C4F58
:1010B0005D8D08CF8280B7170240984F1345F5FF2A
:1010C000798D88CF828099C5371702405C4F5D8D3E
:1010D00048CF8280B7170240D84F1345F5FF798D6E
:1010E000C8CF828099C5371702405C475D8D48C7DD
:1010F0008280B7170240D8471345F5FF798DC8C7DE
:101100008280EFF24FC11629F577FD17F58FF62192
:10111000DA257971D58F1EA95625FD779387379FDC
:10112000F58FD6212A842EC6D58F9625D58FB62544
:10113000D58F5EA55E29C207C18393F7F7CFD98FFC
:101140005EA96808C13BB747014093870780B24555
:10115000631EF402A2576547B387E70298419306DE
:1011600040060A07B3D7E70233D7D702B3F7D7024F
:101170001207920793872703B3D7D702BD8BD98F66
:10118000C207C1831EA445616FF02FBB9257E1B720
:1011900091C55E250967D98F5EA582805A25F977AA
:1011A000FD17F98FD5BF13F7F50F85471583B39555
:1011B000B7006319F7009307C500984301CED98D96
:1011C0008CC38280894693074501E318D7FE9307B5
:1011D0000501E5B793C5F5FFF98DDDB793F5F51F6B
:1011E0004EA182804A211375F51F82800A216D8DE0
:1011F0003335A000828013F7F50F85461583B3972A
:10120000B6006311D7025A25F98F1A21014542070A
:10121000418381CB0545A181B315B5006D8F333571
:10122000E000828089466314D7001A29F1BF5A2949
:10123000E1BFB7070020938747249843636FA70255
:10124000D043B386C7006316D50054413E85B2969D
:10125000D4C35041B306C500631CD700B7060020B5
:1012600083A6C6226306D70054431843B29654C1DE
:1012700018C16303F50088C38280BA877DBFEFF28F
:10128000EFA741112AC6EF10C009B706002083A7B7
:10129000C622370600209386C6221306062332454F
:1012A000A1EF370700209307073493F5F7001307E2
:1012B000073481C51387F700419BB705002093854C
:1012C000452423A2050098C19965C115AE97C19B1D
:1012D00023A2070023A00700B385E7409CC21CC3DC
:1012E000B707002023ACB722B707002023AAB722F4
:1012F000B70700804CC31CC2032A0600B377AA00BC
:1013000085E39307F5FF3957636CF70093070501F1
:1013100013F7F70041C313F707FF410763EBE70635
:10132000814489A022872E8461A058C15CC01137F6
:101330005840B7060020938686239042B307E940C1
:1013400023A0F90063F3C7009CC2B70700203367EE
:10135000EA009387C72358C09843C10423200400A0
:10136000050798C3EF10E01893F7F400D1CBA167FD
:101370009387078073900730376600003765000059
:101380001306C66D9305001113054570EF40A009C3
:1013900001A0BA8737070020032947239309472371
:1013A000E360F9F837070020032447241307472494
:1013B00050406374F6000C40B5F59442E38286F623
:1013C0001440044314C33307F64093060002E3F1CC
:1013D000E6F63305F4009376F500A1DAA16793876A
:1013E00007807390073037660000376500001306EA
:1013F000C66D9305F00C13054570EF40C00201A0C7
:10140000268541016FF0CF9255C1EFF2CF90B7071B
:101410000020032745FF83A707232A84B376F7001C
:101420009DE2A167938707807390073037660000BD
:10143000376500001306C66D93054012130545700D
:10144000EF30707E01A0832605FF9DC2A1679387C0
:101450000780739007303766000037650000130679
:10146000C66D9305501213054570EF30D07B01A077
:1014700093C7F7FFF98F232AF5FEEF00906AB707AD
:101480000020938747239443032744FF130504FF59
:10149000369798C3793BB707002093870724984372
:1014A000050798C3EF10E0046FF02F898280B7E73B
:1014B00000E041572387E7402386E740B7F700E085
:1014C00023A0070023A20700814694C70147D8C77D
:1014D00037070020832507201307401F814633D696
:1014E000E5023D4790CBD4CB98C38280EFF2AF8228
:1014F000411102C6F32750303EC6B2470D478D8BCF
:101500006384E702A167938707807390073037668B
:10151000000037650000130686729305600B130503
:101520004570EF30507001A0B78700209387070007
:10153000BD8B9DC3A1679387078073900730376683
:10154000000037650000130686729305B00B130583
:101550004570EF30506D01A0993FB7E700E0056797
:1015600023A0E710116723A0E71023A40180EFE078
:101570003FD9014541016FE05FFC73110134A16760
:101580009387078073900730B7F700E023A2070026
:10159000EF00705B11C5B7E700E0116723A0E720FB
:1015A000A1679387878873900730731101347300A4
:1015B0002030A167938707807390073093878180DD
:1015C0009843050798C38280138781801C438DE769
:1015D000EFE27FF4A1679387078073900730376647
:1015E000000037650000130686729305201013056E
:1015F0004570EF30506301A0FD171CC391E7A16750
:101600009387878873900730828021651305058052
:101610007315053082807310053082809307850032
:101620007D575CC118C55CC51CC92320050082809C
:101630002328050082809841FD5693078500631E8C
:10164000D7001C49D843D8C10CC79CC5CCC31C418A
:1016500088C985071CC18280B687D4439042E37D48
:10166000C7FECDB7544118451C4998C654C3D4434E
:101670006393A600D8C39843232805007D1798C319
:1016800088438280EFE23FE941112AC61D37324587
:10169000005D1D3F1335140041016FE01FEAEFE2CA
:1016A0009FE732893041045D2A8409EE1C410145DF
:1016B00091E70844EF10003523240400850404DC7E
:1016C0006FE0BFE7631009024841EF30B04A5C4069
:1016D00038400145BA9718445CC0E3E1E7FE1C407E
:1016E0005CC0E9BF4845EF30F0483C4058441440E6
:1016F000B307F0403E9758C46375D7001844BA97B3
:101700005CC489470145E31BF9FACDD8FD147DB7C8
:10171000EFE2DFDE204541112AC605E4A167938789
:1017200007807390073037660000856537650000D5
:1017300013060675938555BD13054570EF30B04E01
:1017400001A0185C5C5C6365F702A1679387078062
:101750007390073037660000856537650000130613
:101760000675938565BD13054570EF30D04B01A01C
:10177000185C01496378F7028344540401466C0005
:101780002285313F9399840193D98941FD572A8954
:10179000639EF9005C5099C713054402EF1060077F
:1017A00011C105494A8541016FE09FD89307F007B1
:1017B0006395F902A16793870780739007303766B6
:1017C000000085653765000013060675938565BFC3
:1017D00013054570EF30304501A08504E204E18433
:1017E000A3029404C1B7304115C2EFE2DFD25845DD
:1017F0001445AA87329758C56364D700184158C565
:101800002E85CC47EF3010376FE03FD38280EFE278
:101810009FD02A84793B8344540413094402E20490
:10182000E18463459002FD57A302F404713B5133F8
:101830008344440413090401E204E18463499002EF
:10184000FD572302F40449336FE03FCF3C4491CB72
:1018500022857D3D19C1EF106018FD14E204E1847A
:10186000C9B75C50E9D34A85EF00B07AE5B71C48A8
:10187000E1DB4A85EF00F07919C1EF102016FD1465
:10188000E204E18465BFEFE21FC941111DE1A167D8
:101890009387078073900730376600003765000034
:1018A000130606759305001113054570EF30B03728
:1018B00001A05C5D2EC62A84BDC33841B3B7E702E0
:1018C000B9EFC5393040585C1440232C0402B307EB
:1018D000E602B24554C03387F600918FB6975CC4D8
:1018E000FD572302F40418C4A302F40495E11C4834
:1018F00099CB13050401EF00D07111C5B7E700E0E3
:10190000116723A0E720C931054541016FE0FFC2FF
:10191000130504012133130544020933EDB7A16710
:1019200093870780739007303766000037650000A3
:10193000130606759305501413054570EF30B02E4D
:1019400001A0EFE25FBD411139C1B3B7A502AA847E
:101950009DEF3305B502930730FB63EAA702130539
:10196000C5042EC6EFF0BF912A8411CDB245AA87D7
:1019700099C19307C5042CC01CC044DC8545228551
:10198000193723240404228541016FE01FBBA1679E
:101990009387078073900730376600003765000033
:1019A000130606759305601C13054570EF30B027CC
:1019B00001A0EFE2DFB3011132C61DE1A1679387F9
:1019C0000780739007303766000037650000130604
:1019D00006759305E03213054570EF30D02401A061
:1019E0002A842E89B6848DE53C419DC3A1679387E7
:1019F00007807390073037660000376500001306D4
:101A000006759305F03213054570EF30D02101A023
:101A100089476398F402585C85476304F702A1671D
:101A200093870780739007303766000037650000A2
:101A3000130606759305003313054570EF30B01E8D
:101A400001A0EF00707A15E5B247014C85C7A16788
:101A50009387078073900730376600003765000072
:101A6000130606759305303313054570EF30B01B30
:101A700001A0014C094BFD59930B040137EA00E02A
:101A8000916AA5A85C50C5C313054402EF007058C5
:101A900059A8B24781E70D3E014571A863150C00B6
:101AA0002808EF00D0650D36EF00B00719368347E0
:101AB0004404E207E1876394370123020404834767
:101AC0005404E207E18763943701A3020404ED3C68
:101AD0006C002808EF0010643DE9E13C185C5C5C98
:101AE000631EF704D534B2455E85EF00B04622850B
:101AF000393BEF00102029C9054C653C185C5C5C43
:101B00006364F700E39764F92686CA8522858329F2
:101B1000840371363C44BDD789476394F400639ACB
:101B200009002285F53611C5B7E700E0116723A04B
:101B3000E720593C054505616FE0FF9E7134228521
:101B4000F931EF00101B4DBF23205A2175B72285B4
:101B50007D39EF00101A89B7EFE25F9A41111DE15C
:101B6000A167938707807390073037660000376559
:101B70000000130606759305204013054570EF30ED
:101B8000900A01A02A84328A36898DE53C419DC3A2
:101B9000A167938707807390073037660000376529
:101BA0000000130606759305304013054570EF30AD
:101BB000900701A089476318F902585C85476304C0
:101BC000F702A1679387078073900730376600009C
:101BD00037650000130606759305404013054570F0
:101BE000EF30700401A02EC6EFF03FA2185C5C5CE1
:101BF000AA8AB2456366F700894781446318F902EF
:101C0000834454044A86228593998401032B8403D8
:101C1000793493D98941FD576391F9043C449DC7B8
:101C20008947631CF900630A0B0085445685EFF071
:101C30009F9E268541016FE0BF8F2285D13C75D5DF
:101C4000E3050AFE85472320FA00C5B75C50F1DFA3
:101C500013054402EF00F03BDDB79307F0076394F0
:101C6000F902A167938707807390073037660000F9
:101C700037650000130606759305D04813054570B7
:101C8000EF30607A01A08504E204E184A3029404A9
:101C900069BFEFE2DF85011132C61DE1A1679387BD
:101CA0000780739007303766000037650000130621
:101CB00006759305105513054570EF30C07601A0E9
:101CC0002A84AE898DE53C419DC3A1679387078037
:101CD00073900730376600003765000013060675FD
:101CE0009305505513054570EF30E07301A0EF00E8
:101CF000B04F15E5B247014985C7A16793870780B3
:101D000073900730376600003765000013060675CC
:101D10009305A05513054570EF30E07001A001490F
:101D20007D5A930A440237EB00E0916B85A8B247D5
:101D300089E7EFF07F89014559A863150900280854
:101D4000EF00F03BEFF05F88E92BEFF09F868347D1
:101D50004404E207E18763944701230204048347B4
:101D60005404E207E18763944701A3020404EFF0FF
:101D7000BF856C002808EF00F0393DE12285EFF0C7
:101D80007F9029C9B2455685EF00D01C2285413489
:101D9000EF00207619E123207B210549EFF07F81B8
:101DA000045CD1D4CE852285FD14EFF0DFA304DCE2
:101DB0001C4899CB13050401EF00B02511C5B7E706
:101DC00000E0116723A0E720EFF01F8005450561C3
:101DD0006FE06FF52285EFF09FA3EF00807175BF74
:101DE0002285EFF0DFA2EF00C0702285EFF09F891F
:101DF0004DD591B7EFE22FF241111DE1A167938715
:101E000007807390073037660000376500001306BF
:101E100006759305407F13054570EF30C06001A043
:101E20002A84EFF00FF91C5C485C1D8D2AC6EFF088
:101E3000AFF9324541016FE04FF015E5EFE2AFED4C
:101E4000A167938707807390073037660000856528
:101E50003765000013060675938585AC130545703C
:101E6000EF30605C01A09DCD3766002093060634FC
:101E70008147014713060634214883A8460063982A
:101E8000A80093173700B2978CC3C8C321A891E765
:101E900083A8060063930800B6870507A106E31E22
:101EA00007FDFDF38280EFE20FE741112A842EC681
:101EB00032C4EFF00FF0834744047D572246E20717
:101EC000E187B2456394E700230204048347540486
:101ED0007D57E207E1876394E700A302040432C65A
:101EE0002EC4EFF06FEE1C5CA245324689E7130565
:101EF0004402EF00B00A2285EFF07F9141016FE0CC
:101F0000CFE3EFE24FE101469145EFF09FA36FE091
:101F1000CFE2EFE24FE041112AC62EC4EFF06FE9A5
:101F20003245A24501443C4591E71C5D014499E3DB
:101F30002CC50544EFF04FE9228541016FE0EFDF4A
:101F4000EFE26FDD41112E866C0002C699333245F7
:101F500041016FE08FDE37070020130707251C4380
:101F60009443B70700209387072781E67D5798C3DE
:101F70008280184358471843DDBFEFE22FD8370956
:101F80000020B70700209304C92483A907282A84C6
:101F90009C4088404111A388070411052EC6EFF02C
:101FA0006FEC7D579307C924B245631CE40295C9C1
:101FB000B7670020938707429440D84398C61047DC
:101FC0009440D0C694401047910654C29440910664
:101FD00014C798405CCB9843050798C341016FE054
:101FE0002FD598434E9440C3637B340137070020BC
:101FF000032547258C439105EFF0EFE3C5B737077D
:102000000020032507258C439105EFF0CFE2B707A9
:102010000020938707279843E372E4FC80C37DBFC9
:10202000EFE2CFCD37640020B7090020130444430A
:10203000370A00209384C9259C40EDDFEFF06FD76D
:102040005C4403A9C70013054900EFF0AFE1130793
:102050008A251C43FD171CC39C40FD179CC0EFF054
:10206000AFD603250903EFF02FBA4A85EFF0CFB9B9
:10207000D1B7EFE2CFC713192600AA8A4A85AE89E5
:10208000368BBA8B3E8AEFF08F9F1DC1AA84130551
:102090004005EFF0CF9E2A8409C904D98147C14683
:1020A000639A0900230A050225A02685EFF0CFB523
:1020B0007D55D1A23387F900030707003306F400EA
:1020C000230AE60201C78507E396D7FEA3010404AD
:1020D000914763F47703A167938707807390073074
:1020E00037660000376500001306467693057039A1
:1020F00013054570EF30203301A0930944004E854D
:10210000232674032322740523240404EFF04FD202
:1021100013058401EFF0CFD115471305C9FF33072D
:102120007741269500C818CC40D023060404A306A6
:10213000040423070404A307040423080404A308D5
:1021400004045A86D6854199EFE08FAB08C063043A
:102150000A0023208A00EFF0CFC5B707002093873D
:10216000872598433709002037650020050798C365
:102170001307C9241843370A00201309C9249304FC
:102180000538130ACA27631A070E232089009843CB
:1021900085476310F70813050538EFF02FC813853E
:1021A0004401EFF0AFC713858402EFF02FC713850A
:1021B000C403EFF0AFC613850405EFF02FC63765F3
:1021C0000020130B453E1305453EEFF02FC5376544
:1021D0000020930A853F1305853FEFF02FC4376534
:1021E00000201305C540EFF06FC3376500201305CD
:1021F0004543EFF0AFC23765002013050542EFF00D
:10220000EFC1B707002023A86725B707002023AA3E
:102210005725B7070020938747269843050798C39B
:1022200037070020130787265C54144363F3F60036
:102230001CC35147B387E702BE94DC4098471CC4D7
:1022400058C498472322370123A437019C4044C82F
:1022500085079CC0EFF04FB783270A00054581CF63
:1022600083270900D8575C546377F700B7E700E08D
:10227000116723A0E7206FE00FAB83270A00D1FB93
:1022800083270900D8575C54E3E5E7F82320890049
:1022900049B7EFE24FA8B7070020B7650000372520
:1022A00000009387C72601478146130600109385D7
:1022B000857713050502753B0544631E8502EF0013
:1022C000302E631A8502A1679387078073900730C9
:1022D000B70700207D5723A8E726B707002023AEC5
:1022E000A726B707002023A00728EFF02FA083A779
:1022F000C1806FE08FA4FD57E31BF5FEA1679387B4
:1023000007807390073037660000856537650000E9
:10231000130646769385058413054570EF30A010AB
:1023200001A0B7070020938707269843050798C3A5
:102330008280B707002003A507288280B707002006
:1023400003A507288280B707002083A70726639983
:102350000718EFE24F9CB7070020938707288043B8
:10236000050480C321ECB707002093870725984315
:10237000184305C7A16793870780739007303766B6
:10238000000085653765000013064676938575ACB9
:1023900013054570EF30200901A03707002013070F
:1023A00047259443104390C3B707002014C3938775
:1023B00047279843050798C3EFF0FFB93706002079
:1023C000930706279C4337670020B70500201306B4
:1023D0000627130707389385C52401456375F40262
:1023E0009C41D146DC57B387D7023E9718438547B7
:1023F00063F3E7000545B707002083A7472891C38B
:1024000005456FE08F93370E0020B70E0020514F27
:1024100093070E259443944281E6FD571CC2C9B729
:102420009C43DC47DC47D4436374D40014C24DBFE3
:1024300083A8870003A8C700D44B1383470023A4B5
:1024400008012322180183A846006394680023A290
:10245000060103A8060023AA07007D1823A0060191
:10246000945795CA03A8C70183A8070283AF460003
:102470002324180183A8070223A2080113888701D7
:1024800063940F0123A2160103A8060023A40702E8
:102490007D1823A0060193868E2603A8C70283A871
:1024A000060063F4080123A00601B306E803BA9608
:1024B00083A8460083AF880023A4170123A6F70151
:1024C00083AF880023A26F0023A46800D4CB9C4272
:1024D00085079CC29C41DC57E36CF8F205450DBFB3
:1024E000B70700209387872798430145050798C3BE
:1024F0008280EFE2AF8037040020130404261C40E2
:10250000411185E7A167938707807390073037668D
:102510000000856537650000130646769385358B88
:1025200013054570EF20307001A0EFF08F881C403C
:10253000FD171CC01C4089CB01452AC6EFF0CF888F
:10254000324541016FD0DFFEB707002083A7872502
:10255000E5D7B76600203765002081479386C640DF
:10256000370F002013050538D14837030020370EF8
:102570000020854E59A8DC46DC47CC4F9053985735
:1025800090C503A807022322B800032847009385BB
:1025900087016313B80050C3104323A407027D16BC
:1025A00010C38C47D047D84B1388470090C54CC206
:1025B0004C436393050150C3104323AA07007D16C3
:1025C00010C313078F26D0570C4363F3C50010C305
:1025D000330716032A974C4383AF85008CC723A685
:1025E000F70183AF850023A20F0123A405010C434B
:1025F000D8CB85050CC31307C3241843585763660B
:10260000E60013074E282320D70198422DF799C3DF
:10261000EFF07F94B70700201387872704431384C4
:10262000872791CC370900208549313B09C593079D
:10263000492823A03701FD14EDF823200400B70733
:10264000002083A74728E38907EEB7E700E011677A
:1026500023A0E7200545D5B519E5B7E700E01167E8
:1026600023A0E7208280EFD21FEBB707002083A7CB
:10267000072641119DC3A167938707807390073098
:1026800037660000376500001306467693059054C0
:1026900013054570EF20305901A02AC65931324543
:1026A0008145EFF09F8DB13511E5B7E700E0116787
:1026B00023A0E72041016FD05FE8B707002003A700
:1026C0000726B70700209387472801C7054798C307
:1026D000828023A00700B7070020138787261843AE
:1026E00013868726B7670020938707385148B306BB
:1026F0000703B385D700884115C5C841A106BE961A
:102700004841C8C16314D5005441D4C1D146B30671
:10271000D702B697DC43D447B707002023A6D724B7
:1027200018C2828015E7EFD21FDFA1679387078069
:102730007390073037660000856537650000130623
:102740004676938525C013054570EF20D04D01A036
:102750007D1771BFEFD23FDC05E5A1679387078046
:1027600073900730376600008565376500001306F3
:1027700046769385C5C113054570EF20D04A01A068
:10278000B70700202E8483A5C724E105EFE0BFEA48
:1027900085452285EFF06FFE6FD03FDAEFD2BFD7CD
:1027A0002A8705E5A167938707807390073037660E
:1027B000000085653765000013064676938525C5BC
:1027C00013054570EF20304601A0B707002093871E
:1027D000C72454432E858C4303A88600D4CD8C4354
:1027E00023A0050303A807008C46610823A2050166
:1027F00003A807009C43610823A4060198D71C4343
:1028000085071CC311C27D55B285EFF00FF76FD05D
:10281000DFD25C45DC4795E7EFD2FFCFA167938716
:1028200007807390073037660000856537650000C4
:1028300013064676938525C813054570EF20B03EF4
:1028400001A0D04F945398579385870114C6D0C2E6
:1028500050436313B60054C3144323A40702FD1668
:1028600014C33707002003270726D45725EF8C47CA
:10287000D047D84B90C5D04748434CC293854700BA
:102880006313B50050C3104323AA07007D1610C37D
:10289000370700201307872610436373D60014C33D
:1028A00051473386E602376700201307073832970F
:1028B0005043084690C7C8C708464CC10CC6D8CB81
:1028C0001C43014585071CC3B707002083A7C72405
:1028D000DC5763F8D700B7070020054723A2E72895
:1028E00005458280376700201307C74050430846DC
:1028F000D0CF88D308464CC10CC698D7D1B7B707FC
:10290000002083A747271CC1B707002083A70728FB
:102910005CC18280EFD23FC0411105E5A16793877A
:1029200007807390073037660000856537650000C3
:10293000130646769385D5CF13054570EF20B02E4C
:1029400001A085E5A16793870780739007303766FC
:102950000000856537650000130646769385E5CF50
:1029600013054570EF20302C01A02EC62AC4EFE0DD
:102970005FC437070020B70700201307C72483A6CA
:1029800007281C432245B24583C7170599CB1C4332
:10299000A38807040544EFE03FC3228541016FD0BF
:1029A000DFB99C417D570144E387E7FE37060020ED
:1029B000032646270328050058416307C80063E53E
:1029C000E60023A00500F9B73386E640E37BF6FE78
:1029D000958FBA979CC12537014475BFB707002072
:1029E000054723A2E7288280B707002083A7C727CF
:1029F000054581CBB707002003A507261335150031
:102A00000605828011E50145828001456FD0FFB245
:102A1000EFD27FB0B707002083A7C7242A8463853D
:102A2000A702A1679387078073900730376600007D
:102A3000856537650000130646769385F504130512
:102A40004570EF20501E01A0BC4785E7A167938722
:102A50000780739007303766000085653765000092
:102A6000130646769385050513054570EF20B01BC8
:102A700001A054557841FD173CC5E388E6F8D1F72D
:102A8000930445002685EFE0FFBD7C4015471D8F70
:102A900018CC370700201307872614435CD463F350
:102AA000F6001CC351473387E702B76700209387BE
:102AB00007380545BA97D843144718C454C4144777
:102AC000C4C204C798435CC8050798C381B7EFD256
:102AD0009FA437040020EFE0DFAD130444291C401D
:102AE000B1E7376500201309854413058544EFE0FD
:102AF000FFB2376500209304C5451305C545EFE0D7
:102B0000FFB1B707002023A427290146B7070020FB
:102B1000C145114523A69728EFE0BFE208C019C5BB
:102B2000B76500009385457AEFF02FB1EFE0DFA99C
:102B30006FD0BFA0EFD23F9E4CC108C9AA87636285
:102B4000B602184D158E0545637BE6009385470058
:102B5000B707002003A5C728EFE0FFAD01456FD000
:102B6000DF9D6375D6000545E3FBD5FE93854700E1
:102B7000B707002003A58728C5B7EFD2DF992A84BD
:102B8000AE8432890C4CA6864A86A69522855D378E
:102B900019E16FD09F9A1C4C2285BE941C508297DD
:102BA000D5B7EFD25F97B707002083A787284111D9
:102BB000AA84DC472EC6C04713054400EFE09FAA55
:102BC00083474402324613F7470011CBA68522857E
:102BD0006D371C502285829741016FD01F96F99B5B
:102BE0002302F402FDB7EFD21F93370400209306AF
:102BF000842898421C4391EBB70700209387C7288D
:102C0000904398C390C26FD05F935C47FD55884353
:102C1000493FF1BFEFD2BF8D19694111B70A0020BA
:102C2000B7090020370B0020B70B002013090978E3
:102C300083A78A28984329CBDC47814C03AC070043
:102C4000EFF02FEEEFF0EFEE83A709292A849384AB
:102C50000929130A4B29636CF50288C0638F0C02A3
:102C600083A7CB2890431336160003250A00B3052B
:102C70008C40EFF04FA3EFF0DF8711EDB7E700E0F6
:102C8000116723A0E72001A8854C014C55BFA13F47
:102C900080C0EFF01F86214C05A00146E36785FD4B
:102CA000EFF03F85A2856285ED3DF5B79247B245CD
:102CB0008297824763DD070003250A0001468A8563
:102CC000EFE03FFD35D582472245E3C107FE2244B0
:102CD0005C4895E3EFF0EFE59C40AA8C6373F50048
:102CE0001937824723A09401FD17E367FCFC8A078C
:102CF000CA979C43828713054400EFE0BF96D9BF73
:102D0000834744020C4C924693E717002302F402D7
:102D10006686B6952285393D45D18347440213F72F
:102D2000470019CB1C4C924566862285BE95B1356D
:102D30001C502285829749B7F99B2302F402CDBF2C
:102D400083474402F99B2302F402BDB78347440240
:102D5000924593E717002302F4020CCC9DE1A16792
:102D6000938707807390073037660000376500004F
:102D70001306C67A9305903513054570EF20A06AB7
:102D800001A0E6866686E69522856D3335B78347D2
:102D9000440213F727005DF72285EFE0EFE629BF35
:102DA000EFD26FF7EFF0BFD2B707002083A7472914
:102DB0009DE3A16793870780739007303766000013
:102DC000376500001306C67A930590111305457008
:102DD000EF20606501A0B7070020B7650000373518
:102DE00000009387872911478146130600109385B9
:102DF000457C130545C1EFF0CFA745DD6FD0EFF35C
:102E0000EFD26FF101111DE1A167938707807390E5
:102E1000073037660000376500001306C67A930551
:102E2000B01813054570EF20006001A037040020A2
:102E3000130444291C403AC62A8801458DC7B68828
:102E40002EC832CA42CC954663C2B602EFF0DFB953
:102E50003247894781463A866303F50001460840B8
:102E60000C08EFE01FB505616FD02FED8146468657
:102E70000C083E85EFE05FCEFDB7B707002083A7C3
:102E8000072037177A0013070720B3D7E702370761
:102E9000002093F7F70F230FF7281307803EB3871F
:102EA000E70237070020231EF7288280EFD2AFE623
:102EB0002A841165011185451105EFE0EF9E930706
:102EC00000207C82371501408D473EC44C00E1470D
:102ED000130505803EC6EFD0DFEF22C8374401401E
:102EE000B70708000C08130504803ECC02CA231E55
:102EF0000100EFE00FA1854513050480EFE04FA925
:102F000005616FD08FE3EFD26FDFB7440140AE8928
:102F10003289014493840480634524014A856FD03B
:102F20002FE1930500042685EFE04FAC7DD9B387F0
:102F300089008385070026850504C205C181EFE06D
:102F4000EFA9D9BF138701811C43B7760020938670
:102F500086DD3E95636BD500B7860020938606809C
:102F600063E5A60008C33E858280FD57EDBF23269A
:102F700005000CC150C123240500054582805C4535
:102F8000544118458507B3E7D702638EE7005845DB
:102F90001C41BA978CA35C4558418507B3E7E7020B
:102FA0005CC5054582807955828018455C45630F74
:102FB000F70018451C41BA979C239CA11C45584119
:102FC0008507B3E7E7021CC505458280014582807D
:102FD000EFD26FD479711306000281450808EFD053
:102FE0008FD68545114502C202C402C6EFE0CF8BE1
:102FF000854513050020EFE02F8B1165EFD07FF0A2
:10300000371401408547130504804C007C8202C6BA
:10301000EFD03FDCC147130504804C007C8202C620
:10302000EFD03FDB930700024C00130504807C8245
:103030003724014002C6EFD0DFD913050440EFD09A
:103040003F8E85473ECA3ECCB7070E003ECE0C08E9
:103050008D47130504402302F10202C802D0EFD0CD
:103060001F90854513050440EFD0DF958545130576
:103070000440EFD03F94814513050440EFD0FFA4F6
:1030800013050440EFD03F95930404402685EFD00C
:103090003F956DFD1305044037240140EFD0DF94C8
:1030A000930404402685EFD0DF946DFD13050440A2
:1030B000EFD03FA3B70700202390A72A45616FD028
:1030C000CFC7EFD24FC579711306C00281454800C2
:1030D000EFD06FC785450545EFD03FFB3704024071
:1030E00013058400EFD07FB3B72701409387C7440F
:1030F0003EC2B70700209387472A3EC48D473EC88B
:10310000930700083ECC930700103ECE9307004083
:103110003ED0930700023ED24C008D671305840019
:103120003ED402C602CA02D6EFD0FFC545616FD0B9
:10313000CFC0EFD24FBE3705024085452105372469
:103140000140EFD0DFC7130504409D460546814589
:10315000EFD03F8C130504409D4609469145EFD0C2
:103160005F8B9D460D46130504409545EFD07F8A41
:10317000130504408545EFD0FF84854513050440C1
:10318000EFD0BF876FD06FBBEFD2EFB8411185454D
:1031900013050004EFD05FF1A147372401407C8282
:1031A00085473EC44C00C147130504803EC6EFD09E
:1031B0005FC2014613050480A145EFD03FCE914781
:1031C0004C00130504807C82EFD0BFC0014613057C
:1031D00004809145EFD09FCC930700084C00130565
:1031E00004807C82EFD0FFBE014613050480930566
:1031F0000008EFD0BFCA930700104C0013050480ED
:103200007C82EFD01FBD014613050480930500109A
:10321000EFD0DFC8930700204C00130504807C82A8
:10322000EFD03FBB01461305048093050020EFD08B
:10323000FFC6930700404C00130504807C82EFD04A
:103240005FB901461305048093050040EFD01FC508
:103250008567938707804C00130504807C82856412
:10326000EFD03FB701469385048013050480EFD06B
:10327000FFC24C00130504806482EFD09FB5014665
:10328000130504808565EFD07FC189644C00130568
:1032900004806482EFD0FFB3014613050480896582
:1032A000EFD0DFBF91674C00130504807C82EFD024
:1032B0005FB20146130504809165EFD03FBEE17710
:1032C0004C00130504807C82EFD0BFB0014613058B
:1032D0000480A165EFD09FBC4C003715014064828B
:1032E000EFD03FAF0546896537150140EFD01FBBD2
:1032F00041016FD08FA4EFD20FA2EFD03FBA6FD0B1
:10330000CFA3EFD24FA1EFD0DFB86FD00FA3EFD292
:103310008FA079712A89854513050004EFD0DFD885
:1033200037240140930700028D44FC824C08C147BA
:10333000130504803ECE26CCEFD0BFA9014613056D
:10334000048093050002EFD07FB585454145EFD05D
:10335000BFD5854513050004EFD0FFD68547FC8215
:103360004C08E1473715014026CC3ECEEFD07FA672
:103370008947FC824C0891473715014037240040AB
:103380003ECEEFD01FA50C10B7070C00130504802C
:103390004AD03ED402D223160102EFD09FD6930723
:1033A00070357C86680085473EC84487EFD05FB0A3
:1033B00013050480054693055052EFD0DFDE054625
:1033C0001305048093054042EFD0FFDD85451305CA
:1033D0000480EFD0FFDB45616FD02F96EFD2AF9323
:1033E00079712A89854513050004EFD0FFCB372476
:1033F0000140930700048D44FC824C08C14713052B
:1034000004803ECE26CCEFD0DF9C0146130504801D
:1034100093050004EFD09FA885454145EFD0DFC854
:10342000854513050008EFD01FCA9147FC824C0860
:10343000E1473715014026CC3ECEEFD09F99A147FA
:10344000FC824C08914737150140372400403ECE9E
:10345000EFD03F980C10B7070C00130504C04AD0FA
:103460003ED402D223160102EFD0BFC993078035A4
:103470007C86680085473EC84487EFD07FA313054C
:1034800004C0054693055052EFD0FFD10546130501
:1034900004C093054042EFD01FD18545130504C0F9
:1034A000EFD01FCF45616FD04F89EFD2CF867971B2
:1034B0002A8985451145EFD03FBF37140140894720
:1034C0008D44FC824C08C147130504803ECE26CCB7
:1034D000EFD03F900146130504808945EFD01F9C33
:1034E00085451145EFD05FBC854537050200EFD01B
:1034F0009FBD9147FC824C08E1471305048026CC10
:103500003ECEEFD01F8DA147FC824C08914713059A
:1035100004803ECE37440040EFD0BF8B0C10B7077D
:103520000C00130504404AD03ED402D223160102F7
:10353000EFD03FBD930760337C86680085473EC867
:103540004487EFD0FF96130504400546930550527B
:10355000EFD07FC505461305044093054042EFD0E8
:103560009FC4854513050440EFD09FC245616FC0DD
:10357000DFFCEFC2BFF87971AA8985452145EFD0FC
:10358000BFB23719014085470D44C1444C081305AB
:1035900009C0FC8226CE22CCEFD0BF8301461305A2
:1035A00009C08545EFD09F8F85454145EFD0DFAFFE
:1035B000854513050010EFD01FB1E1474C083715C2
:1035C0000140E48222CC3ECEEFD0BF8093070002C0
:1035D000FC824C089147371501403ECEEFD06FFF7B
:1035E0000C10B7070C00372500404ED03ED402D255
:1035F00023160102EFD0FFB0930790357C86680058
:1036000085473EC84087EFD0BF8A05469305505294
:1036100037250040EFD03FB9054693054042372596
:103620000040EFD05FB8854537250040EFD05FB64A
:1036300045616FC0FFEFEFC21FEE37140140130565
:103640000440014693050020EFD05F851305044038
:10365000014693050040EFD07F8485650146938540
:10366000058013050440EFD07F836FC01FEDEFC2CC
:10367000FFE879712A8A854513050002EFD0DFA2A1
:103680003714014093070010FC820D49C1474C08D4
:10369000130504403ECE4ACCEFD0AFF301461305EC
:1036A000044093050010EFD06FFF930700204C08F3
:1036B00013050440FC82EFD0CFF1930900404C0881
:1036C00013050440231A31018564EFD08FF04C08B4
:1036D0001305044093840480E482EFD08FEFEFF071
:1036E0009FF585452145EFD03F9C85453705040072
:1036F000EFD07F9DE1474C08130504C0231A310128
:103700004ACC3ECEEFD0EFEC91474C08130504C0F5
:10371000E482375400403ECEEFD0AFEB0C10B70739
:103720000C001305048052D03ED402D223160102AD
:10373000EFD03F9D930770137C8685475C876800B8
:1037400085473EC8EFD0CFF61305048005469305A4
:103750005052EFD05FA50546130504809305404203
:10376000EFD07FA4854513050480EFD07FA245618B
:103770006FC01FDCEFC23FDA37140140130504406D
:10378000014693050020EFD06FF113050440014678
:1037900093050040EFD08FF0856505469385058041
:1037A00013050440EFD08FEF6FC03FD9EFC2BFD6F3
:1037B0003714014013050440014693050020EFD063
:1037C000EFED13050440054693050040EFD00FEDE3
:1037D000856501469385058013050440EFD00FEC05
:1037E0006FC0BFD5EFC23FD337140140130504406B
:1037F000014693050020EFD06FEA1305044005460B
:1038000093050040EFD08FE98565054693850580D7
:1038100013050440EFD08FE86FC03FD2EFC2BFCF97
:103820003714014013050440054693050020EFD0EE
:10383000EFE613050440014693050040EFD00FE684
:10384000856501469385058013050440EFD00FE59B
:103850006FC0BFCEEFC23FCC371401401305044008
:10386000054693050020EFD06FE3130504400146A1
:1038700093050040EFD08FE285650546938505806E
:1038800013050440EFD08FE16FC03FCBEFC2BFC83C
:103890007971AA8485454145EFD01F81854513057F
:1038A0000002EFD07F80854537051000EFD0BF8143
:1038B00085670D44FC824C08E1473715014022CC56
:1038C0003ECEEFD00FD1914737150140FC824C0816
:1038D0009147130505403ECEEFD0AFCFB7070C00A0
:1038E0000C10375500403ED426D002D223160102D8
:1038F000EFD03F8105469305505237550040EFD039
:103900009F8A930750147C86680085473EC840878D
:10391000EFD00FDA854537550040EFD07F874561FE
:103920006FC0BFC1397106DE16DC1ADA1ED82AD67E
:103930002ED432D236D03ACE3ECC42CA46C872C617
:1039400076C47AC27EC0B529F250E2525253C253B5
:103950003255A255125682567247E2475248C24823
:10396000324EA24E124F824F2161730020303971C6
:1039700006DE16DC1ADA1ED82AD62ED432D236D07B
:103980003ACE3ECC42CA46C872C676C47AC27EC01F
:10399000192BF250E2525253C2533255A2551256CD
:1039A00082567247E2475248C248324EA24E124FE8
:1039B000824F216173002030397106DE16DC1ADA7D
:1039C0001ED82AD62ED432D236D03ACE3ECC42CAD7
:1039D00046C872C676C47AC27EC04D2BF250E252FF
:1039E0005253C2533255A255125682567247E2477D
:1039F0005248C248324EA24E124F824F216173008C
:103A00002030397106DE16DC1ADA1ED82AD62ED4FA
:103A100032D236D03ACE3ECC42CA46C872C676C4FE
:103A20007AC27EC02125F250E2525253C25332551F
:103A3000A255125682567247E2475248C248324E49
:103A4000A24E124F824F216173002030397106DE81
:103A500016DC1ADA1ED82AD62ED432D236D03ACE76
:103A60003ECC42CA46C872C676C47AC27EC04525DC
:103A7000F250E2525253C2533255A2551256825658
:103A80007247E2475248C248324EA24E124F824F0E
:103A9000216173002030397106DE16DC1ADA1ED877
:103AA0002AD62ED432D236D03ACE3ECC42CA46C8DE
:103AB00072C676C47AC27EC0EF008073F250E252C2
:103AC0005253C2533255A255125682567247E2479C
:103AD0005248C248324EA24E124F824F21617300AB
:103AE0002030EFC25FA3EFF0AFCEEFF08FDDEFF04D
:103AF0004FE46FC09FA4EFC21FA2EFF0EFE86FC0CA
:103B0000DFA3EFC25FA185472E86930500086307F8
:103B1000F5028947930500106302F5028D4793056E
:103B20000020630DF5009147930500406308F50000
:103B30009547631DF5008565938505803725014010
:103B400013050580EFF02FFB6FC03F9F99478565F8
:103B5000E306F5FE9D478965E302F5FEA147916501
:103B6000E30EF5FCA547A165E30AF5FCA947E31DB3
:103B7000F5FCA145E1B7EFC21F9A05479305000880
:103B80006308E5020947AA87930500106302E5026E
:103B90000D4793050020630DE50011479305004094
:103BA0006308E5001547631DE5008565938505807D
:103BB0003725014013050580EFF0AFF46FC0FF9784
:103BC00019478565E306E5FE1D478965E302E5FEC5
:103BD00021479165E30EE5FC2547A165E30AE5FC75
:103BE00029471305F00FE39BE7FCA145D1B7EFC2CE
:103BF000FF903704002093070402014913040402D4
:103C00001947D4436392A60893094002B3093903C4
:103C1000330A340183470A0095E7AA841385C90053
:103C20002295EFF0CFB4994703258A006390F40200
:103C3000EFF0EFED930740023309F902854722992F
:103C40002300F900330534016FC09F8E9D476395B3
:103C5000F400EFF0AFF8F9BF89476395F400EFF097
:103C6000DF84C9BFA1476395F400EFF09F90D9B7F7
:103C70008D476395F400EFF09F9F6DBF9547E39BE1
:103C8000F4FAEFF0BFC07DB7050993874702E31A46
:103C9000E9F6014555BF814709C91821814711C778
:103CA0005C49084D898FB337F0003E858280EFC2B2
:103CB0009F8641112A84A3070100EFF0DFFD19C59B
:103CC0009305F1001305C400EFF02FAE8887410182
:103CD0006FC0BF86EFC23F84B7070020B7650020E2
:103CE00023ACA70A13060010938505470D45EFF096
:103CF0001FF0B707002023AAA72C6FC01F84EFC2B4
:103D00009F81B7070020B765002023AEA70C1306DC
:103D10000040938505571545EFF07FEDB70700206C
:103D200023ACA72C6FC07F81B707002083A7472C47
:103D30006399A700B707002083C7C72D858B3E85F1
:103D40008280B707002083A7872C6398A700B70756
:103D5000002083C7C72D898BDDB7B707002083A755
:103D6000C72C6398A700B707002083C7C72D918B86
:103D7000F9B7B707002083A7072D6398A700B707F7
:103D8000002083C7C72DA18B5DBFB707002083A785
:103D9000472D6399A700B707002083C7C72D93F766
:103DA000070271BFB707002003A7872D9307F00F05
:103DB000E317E5F8B707002083C7C72D93F707047B
:103DC000BDBFEFC24FF53745004093055052130574
:103DD0000540EFD04FC231C5B70700209387172B9E
:103DE000982309E7054798A3EF00100237450040E4
:103DF00013050540EFD00FBF9375F50FB7070020EF
:103E0000238AB72AB707002003A5C72C1C4D1049E9
:103E100054498507B3E7C7026385D7003105EFF042
:103E20000F96374400409305707213050440EFD09D
:103E30008FBC31CDB707002083A7C72C9633BA3388
:103E400063ECE60201469305707213050440EFD05F
:103E50008FB5B70700209387C72D98236D9B98A334
:103E6000EF00303B371501400146894513050580B9
:103E7000EFD0CF826FC06FECD84F1386160092B38D
:103E8000B307D7008C2313050440EFD02FB5374577
:103E900000409305404213050540EFD0CFB579D9D6
:103EA000EF00A06CC1BFEFC20FE73755004093058C
:103EB000505213050580EFD00FB431C5B70700206D
:103EC0009387972B982309E7054798A3EF0040773E
:103ED0003755004013050580EFD0CFB09375F50F2F
:103EE000B7070020238EB72AB707002003A5472D68
:103EF0001C4D104954498507B3E7C7026385D700B5
:103F00003105EFF0CF8737540040930570721305E9
:103F10000480EFD04FAE25C1B707002083A7472DFF
:103F20009633BA3363EEE6020146930570721305C9
:103F30000480EFD04FA7B70700209387C72D9823A1
:103F40001377F7FD98A3EF00502F37150140014676
:103F50009305001013050540EFC05FF46FC0EFDD5F
:103F6000D84F1386160092B3B307D7008C231305DE
:103F70000480EFD0AFA637550040930540421305AB
:103F80000580EFD04FA779D91D25C9BFEFC2AFD8A3
:103F90009305505237550040EFD0EFA515C937555E
:103FA0000040EFD02FA49375F50FB70700202380B2
:103FB000B72CB707002003A5872D1C4D1049544985
:103FC0008507B3E7C7026385D7003105EFE03FFB04
:103FD0009305707237550040EFD0EFA115C9B707B0
:103FE000002083A7872D9633BA3363E5E6020146A6
:103FF0009305707237550040EFD0EF9AB707002055
:104000009387C72D98231377F7FB98A3EF003024ED
:104010006FC0AFD2D84F1386160092B3B307D70044
:104020008C2337550040EFD06F9BDDB7EFC2AFCE8A
:10403000372500409305505213050580EFD0AF9B04
:1040400029C5B70700209387A72A982301E70547CA
:1040500098A3BD2B3725004013050580EFD08F981E
:104060009375F50FB70700202386B72AB7070020FE
:1040700003A5472C1C4D104954498507B3E7C702D7
:104080006385D7003105EFE09FEF372400409305AB
:10409000707213050480EFD00F9639CDB70700205A
:1040A00083A7472C9633BA3363EDE60201469305A6
:1040B000707213050480EFD00F8FB707002093872D
:1040C000C72D9823799B98A3EF0030123725014024
:1040D00001469305000213050580EFC03FDC6FC069
:1040E000CFC5D84F1386160092B3B307D7008C23E1
:1040F00013050480EFD08F8E372500409305404292
:1041000013050580EFD02F8F79D93129C9BFEFC2B0
:104110008FC03725004093055052130505C0EFD0DE
:104120008F8D29C5B70700209387D72A982301E7E9
:10413000054798A3652937250040130505C0EFD032
:104140006F8A9375F50FB70700202388B72AB70742
:10415000002003A5872C1C4D104954498507B3E75F
:10416000C7026385D7003105EFE07FE137240040C7
:1041700093057072130504C0EFD0EF8739CDB707F0
:10418000002083A7872C9633BA3363EDE6020146FD
:1041900093057072130504C0EFD0EF80B7070020BD
:1041A0009387C72D9823759B98A3EF00500537255B
:1041B000014001469305000413050580EFC01FCEA2
:1041C0006FC0AFB7D84F1386160092B3B307D700AE
:1041D0008C23130504C0EFD06F8037250040930572
:1041E0004042130505C0EFD00F8179D9B12EC9BF68
:1041F000EFC26FB29305505237250040EFC0BFFFAA
:1042000039C1B70700209387572B982301E705474B
:1042100098A3092937250040EFC0DFFC9375F50FFF
:10422000B7070020238CB72AB707002003A5072D66
:104230001C4D104954498507B3E7C7026385D70071
:104240003105EFE0DFD39305707237250040EFC0F2
:104250009FFA31CDB707002083A7072D9633BA33D5
:1042600063ECE60201469305707237250040EFC00B
:104270009FF3B70700209387C72D98235D9B98A3D2
:10428000EF00607A3715014001468545130505C0EA
:10429000EFC0DFC06FC06FAAD84F1386160092B36D
:1042A000B307D7008C2337250040EFC03FF39305B9
:1042B000404237250040EFC01FF469DDC12CD9BF53
:1042C000EFC26FA541112A842EC632C4EFF0DFA5DC
:1042D0002A8941EDB2452246B707002083A4472C26
:1042E0004CCC2310040232B0639E84023725014077
:1042F00005469305000213050580EFC03FBA054649
:10430000930570723724004013050480EFC0BFE9A5
:104310009A30DC4C130504809306170096B0BA97C8
:104320008C2391A0B707002083A4872C6393840477
:104330003725014005469305000413050580EFC0AD
:10434000FFB53724004093057072130504C005467D
:10435000EFC07FE59A30DC4C130504C093061700CC
:1043600096B0BA978C23EFC07FE74A8541016FC0B2
:10437000CF9CB707002083A4C72C639D8402371508
:1043800001400546894513050580EFC03FB137441C
:10439000004093057072130504400546EFC0BFE06E
:1043A0009A30DC4C130504409306170096B0BA9778
:1043B0008C2355BFB707002083A4072D639B84027D
:1043C0003715014005468545130505C0EFC01FADF3
:1043D00093057072372500400546EFC0DFDC9A3048
:1043E000DC4C372500409306170096B0BA978C2313
:1043F0009DBFB707002083A4472D63918402371522
:10440000014005469305001013050540EFC01FA9A4
:1044100005469305707237540040FDB5B70700207C
:1044200083A4872DE39384F493057072375500407D
:104430000546EFC05FD79A30DC4C375500409306F5
:10444000170096B0BA978C2339BFB707002083A70F
:10445000472C6399A700B707002083C7A72A858B3D
:104460003E858280B707002083A7872C6397A7002B
:10447000B707002083C7D72ADDB7B707002083A777
:10448000C72C6397A700B707002083C7172BC1BFAE
:10449000B707002083A7072D6397A700B707002061
:1044A00083C7572B6DBFB707002003A7472D93077E
:1044B000F00FE317A7FAB707002083C7972B45B77C
:1044C000EFC26F8585476318F500238AA180EFF05E
:1044D0008F966FC08F8689476317F500238AA18066
:1044E000EFF04FA9FDB78D476317F500238AA18030
:1044F000EFF0CFABF9BF91476317F500238AA18096
:10450000EFF04FAEF9B795476317F500238AA18006
:10451000EFF0CFB07DBF9947E31DF5FA238AA18064
:10452000EFF04FB37DB7EFB21FFFB707002003A432
:10453000072EEFD0BFE02A860147814699452285A4
:10454000EFE01F8C6FB07FFFEFB2FFFCB7070020DA
:1045500003A4472EEFD09FDE2A8601478146994566
:104560002285EFE0FF896FB05FFDEFB2DFFAB7079A
:10457000002003A4872EEFD07FDC2A8601478146E6
:1045800099452285EFE0DF876FB03FFBEFB2BFF8C0
:10459000B707002003A4C72EEFD05FDA2A860147B1
:1045A000814699452285EFE0BF856FB01FF9EFB2D4
:1045B0009FF6B707002003A4072FEFD03FD82A8625
:1045C0000147814699452285EFE09F836FB0FFF652
:1045D000EFB27FF4B707002003A5072E01478146FD
:1045E0000146A145EFE0DF816FB03FF5EFB2BFF2CA
:1045F000B707002003A5472E014781460146A14584
:10460000EFE01F806FB07FF3EFB2FFF0B70700203D
:1046100003A5872E014781460146A145EFE04FFEE5
:104620006FB0BFF1EFB23FEFB707002003A5C72E71
:10463000014781460146A145EFE08FFC6FB0FFEFD7
:10464000EFB27FEDB707002003A5072F0147814692
:104650000146A145EFE0CFFA6FB03FEEEFB2BFEBFE
:104660002A84EFF06FEC01E92285EFF01FDE33358D
:10467000A0006FB09FEC0545EDBFEFB2DFE9EFF0B2
:10468000AFEA6FB09FEBEFB21FE91305803EEFD0AA
:10469000BFFCE5BFEFB23FE81305007DEFD0DFFBC5
:1046A000E5BFEFB25FE7370400200325842DEF005C
:1046B00030435145EFD05FFACDBFEFB2DFE58D2A31
:1046C000FDBFEFB25FE5716513050520EFF02FE345
:1046D000096513050558EFF0EFDFEFF0CFC1EFF0FC
:1046E0004FC05928B7070020B765000037450000C4
:1046F0009387472F09478146130600209385C57C81
:1047000013054569EFD0FF96B7070020B765000095
:10471000374500009387C72F1147814613060010C5
:104720009385857D1305A56BEFD0BF94B765000019
:1047300037450000938701900D478146130600100E
:104740009385857E1305256AEFD0BF92B7070020B9
:10475000B7650000374500009387872F0D478146D6
:10476000130600109385857F13056568EFD07F9051
:10477000EFD03FB26FB07FDCEFB25FD8014691451A
:104780001545EFD00F9C138B41902320AB000146C1
:1047900091451545EFD0EF9A938A819023A0AA0006
:1047A000014691451545EFD0CF99138AC19023203A
:1047B000AA00014691451545EFD0AF989389019124
:1047C00023A0A900014691452945EFD08F97138971
:1047D000419101462320A90091452945EFD06F96CC
:1047E0009384019288C019451384C191EFD06FF171
:1047F000AA8508C003250B00EFD0AFF10C4003A53C
:104800000A00EFD00FF10C4003250A00EFD06FF043
:104810000C4003A50900EFD0CFEF0C4003250900A1
:10482000EFD02FEF0C408840EFD0AFEE6FB05FD0ED
:10483000EFB2DFCC03A5C191FD55B7090020EFD041
:104840002FF023A2A19203A5892D13848191EFF06B
:10485000DFE20DE903A50192B77400209384049769
:10486000014693850401EFD0CFC285472A89631B97
:10487000F5009C4803A5892D9223CC43EFF05FA45B
:1048800023002401370900200325492CEFF01FDD08
:104890000DE903A54190B77500209389059701465E
:1048A00093850597EFD0EFBE8547AA84631BF5007B
:1048B00083A709000325492C9223CC43EFF05FA086
:1048C00004A0B709002003A5892CEFF03FD90DE91A
:1048D00003A58190B77400209384049701469385C3
:1048E0004400EFD00FBB85472A89631BF500DC40ED
:1048F00003A5892C9223CC43EFF09F9C2300240135
:10490000B709002003A5C92CEFF05FD50DE903A579
:10491000C190B77400209384049701469385840066
:10492000EFD02FB785472A89631BF5009C4403A568
:10493000C92C9223CC43EFF0BF9823002401B70980
:10494000002003A5092DEFF07FD115E903A5019102
:10495000B77400209384049701469385C400EFD078
:104960004FB385472A89631CF500D8449C4403A5AE
:10497000092D1223CC43EFF0BF9423002401370903
:1049800000200325492DEFF07FCD31E903A54191AA
:10499000B774002093840497014693854401EFD0B7
:1049A0004FAF8547631DF502DC488823EFF05FB108
:1049B000DC483775000013067009D84394478545D5
:1049C00013058580EF003026DC480325492DD223CE
:1049D0008C47EFF0FF8E230004006FB07FB51C20E2
:1049E000FDFB0D45EFD05FC7FDB7EFB2DFB2B77784
:1049F000002003A50797EFC03FA16FB01FB4EFB22F
:104A00009FB1B777002003A54797EFC0FF9F6FB016
:104A1000DFB2EFB25FB0B777002003A58797EFC092
:104A2000BF9E6FB09FB1EFB21FAFB777002003A555
:104A3000C797EFC07F9D6FB05FB0EFB2DFADB777C4
:104A4000002003A54798EFC03F9C6FB01FAFEFB2A7
:104A50009FACB777002003A50798EFC0FF9A6FB00F
:104A6000DFAD01458280EFB21FAB2545EFF0AF907F
:104A70006FB0BFACEFB23FAA2145EFF0CF8F6FB060
:104A8000DFABEFB25FA91D45EFF0EF8E6FB0FFAA6D
:104A9000EFB27FA81945EFF00F8E6FB01FAAEFB2EB
:104AA0009FA71545EFF02F8D6FB03FA9EFB2BFA6BE
:104AB0001145EFF04F8C6FB05FA8EFB2DFA50D4549
:104AC000EFF06F8B6FB07FA7EFB2FFA40945EFF057
:104AD0008F8A6FB09FA6EFB21FA40545EFF0AF8994
:104AE0006FB0BFA5EFB23FA30C212545EFF06F815A
:104AF00001456FB09FA4EFB21FA20C212145EFF03A
:104B00004F8001456FB07FA3EFB2FFA00C211D4580
:104B1000EFE03FFF01456FB05FA2EFB2DF9F0C21D6
:104B20001945EFE01FFE01456FB03FA1EFB2BF9EF8
:104B30000C211545EFE0FFFC01456FB01FA0EFB25F
:104B40009F9D0C211145EFE0DFFB01456FB0FF9EFB
:104B5000EFB27F9C0C210D45EFE0BFFA01456FB02D
:104B6000DF9DEFB25F9B0C210945EFE09FF9014506
:104B70006FB0BF9CEFB23F9A0C210545EFE07FF884
:104B800001456FB09F9B0145828001458280C167CE
:104B900069768146FD170506139706014183636414
:104BA000B7003E8582803307D5001823B98F21478F
:104BB00013F81700858363050800B18FC207C1830E
:104BC0007D17420741836DF78506F9B7EFB21F9352
:104BD0001389A19283D48192035409008149938758
:104BE000F4FF634CF4029385D4FF377A0020930AD4
:104BF0008A9893F5F50F13058A98EFF05FF9D6942C
:104C000083C7D4FF03C7E4FFA207D98F138701939B
:104C10006318F50095471CC385494E856FB05F91B9
:104C20001306F4FF4206418293851A0013058A9801
:104C3000232007002310C900EF00C073F9BFEFB2B3
:104C40001F8B938401939C403971B1EF03D6A192DD
:104C500085469387A19263F9C60237750020130732
:104C600085980348070093083005930585986310DD
:104C7000180314331307C004639FE650B1479CC068
:104C8000EFD02FEB23A6A19221616FB0DF899308AB
:104C90007004631218510348170013077005631C52
:104CA000E84E94C0F1BF0547138401936396E7046F
:104CB000377700200347A798C1461376F70D63089E
:104CC000D600130707031377F70F63E5E70089475B
:104CD0001CC05DBF9387A1929223232004007D1600
:104CE0004206418292A33775002093058598850579
:104CF00013058598412549BF09476393E70A03D601
:104D0000A19211479386A192E370C7F837750020EE
:104D100093078598B8231308000393058598631FAC
:104D20000701B833DC232207D98F25476369F7428F
:104D300029472394E1928D479CC0B9B74148631B32
:104D40000701B833DC232207D98F25476369F74071
:104D50009D47DDB71308000D63180701B833DC2346
:104D600063EFE73EA547C9BF1308100D6319073F5E
:104D7000D82303C83700220733670701931787003A
:104D80002183D98FC207C1831388F7FF1307E0047B
:104D90006367073D2D4798C0A1072394F192EDB5B5
:104DA0000D476390E70403D6A19299461387A19219
:104DB00063FFC600B776002093868698DC32F42223
:104DC000A207D58FCD4663E7F6009147B5B7914767
:104DD000E3FCC7EA7D16420641822320040012A3A9
:104DE00019B71147639FE7049389A19203D409007F
:104DF000A147E3FB87E803D98192377A0020930A21
:104E00008A989305D9FF93F5F50F13058A98EFF06B
:104E10001FD856998347D9FF0347E9FFA207D98FC7
:104E20006394A700954709BF1306F4FF4206418229
:104E300023A004002390C90093851A0013058A98C3
:104E400055BD15476397E70203D6A19203D7819218
:104E5000377500209387A19293058598631BE632EE
:104E60003387C5008346F7FF59476394E632BD4751
:104E700085B599466395D71EB774002093878498AB
:104E8000B82393070003938484986316F70C03CA2E
:104E90003400DC2003C95400220A336AFA00FC20E3
:104EA0002209130680023369F900420913590941A6
:104EB000931909018145280893D90901EFB0AFE89A
:104EC000930A8101D28B370C0020B3874B41C20774
:104ED000C18363ED370D9109139A190013058A00F8
:104EE000EFC0EFB9930785005CC1930770042ACA2D
:104EF0001CA593077005232045011CB5611A930773
:104F000000033CA5060993578A403CB523062501BA
:104F10001307D500814763CF470B48418609938526
:104F2000D9FF93F5F50F3A9AEFF07FC693578500B6
:104F30002300FA00D947A300AA002301FA0003A521
:104F40000192EFC03FEB01C903A5019281462946BA
:104F50004C08EFC01FA6B820C1476318F70C03CA5E
:104F60003400DC2083C95400220A336AFA00FC2092
:104F7000A2091306800281452808B3E9F900130944
:104F80008101EFB04FDCCA86814789046395F90639
:104F9000D28A370B0020B3874A41C207C18363E638
:104FA00037072320040023950192F9B9130B8C0FC6
:104FB000930C0B0683270B006398770183274B0024
:104FC000014582972390AA00210BE3159BFF890AD4
:104FD000850BE5BD8C0093F6E70FAE9693F51700B1
:104FE0003306F70083D686FD91E1A182850714A2DE
:104FF00093F7F70F0DB7D824D03485072207518FC8
:10500000C2079AA2C183890649B793048B15938B73
:1050100084049C4063955701DC404A858297A10433
:10502000E39974FF0909850ABDB79C341307000D85
:10503000639BE700377500001306A0448545130500
:105040004583D526B9BF1307100DE39CE7F43775E8
:10505000000013064045854513050587DDB71D474C
:10506000639BE70203D6A1921387A192E3FEC6C019
:105070003775002093068598DC32F42293058598D5
:10508000A207D58FCD4663ECF604950786072394D7
:10509000F192914735B921476395E700EFF01FB3CF
:1050A000E5B625476394E7041387A1921223994735
:1050B000E3FCC7BC3775002093058598D6259397E8
:1050C0008600A182D58FC207C1831388F7FF93069C
:1050D000500E63E60601294718C0A9077DB97D1661
:1050E000420641822320040012A311B1294763958F
:1050F000E700EFF0BFAD49BE2D476395E700EFF045
:10510000FFAC59B63147639BE700B777002003C770
:10511000A798A547E3E0E7BCB5475DBE3547639771
:10512000E7049386A19292229147E3FFC7B43775B3
:10513000002093058598D821BC3122075D8F9317F5
:1051400087002183D98FC207C1831388F7FF130714
:10515000F03F63660701394718C099073DB97D16CE
:10516000420641822320040092A251B63947639936
:10517000E7029387A192922303D78192E366E6B078
:1051800037750020930585982E978346F7FF5D4776
:10519000E9B9232004007D164206418292A381BE14
:1051A0003D47E393E7AE3777002093068798DC22EC
:1051B000A83293048798A207C98F13958700A1830B
:1051C000C98F13950701BC22418113061500FD17F5
:1051D00093F7F70F8D4632C63779002063E0F60467
:1051E0002105EFC0CF8932462ACCAA8710C12105FC
:1051F000C8C39305D998812EBC200547639AE7025E
:1052000003A54190EFC01FBFE30D05D803A5419052
:10521000814629462C08EFC0CFF961B33105EFC0B4
:105220000F8632462ACCAA8750C1310588C7D1B72C
:105230000947639EE70003A58190EFC0BFBBE3026F
:1052400005D6814629462C0803A58190E9B78D45EE
:10525000639EB70003A5C190EFC0DFB9E30305D497
:10526000814629462C0803A5C19075B71146639E57
:10527000C70003A50191EFC0FFB7E30405D2814643
:1052800029462C0803A5019179B795466395D70067
:10529000E24798A331A019476390E702E2478CA345
:1052A00003A54191EFC01FB5E30D05CE8146294608
:1052B0002C0803A5419185B79D456395B700E2474A
:1052C00090A3F9BF21466395C700E24794A3C9BFE5
:1052D000A546E38FD7FAE39607CCE247054755BFCB
:1052E000EFB2CFA11384C192AA84EFD08F84032997
:1052F000040023AAA192EFD0CF8333052541930761
:10530000703E9389419363F9A700EFD08F82239574
:10531000019208C023A8019237790020854A114ADA
:10532000130989982685EFE01F97630A55012685A2
:10533000EFE07F9685476319F5026FB06F9FEFC06E
:105340005FFF83A709001D8DE363AAFE9387A192E7
:1053500082232685130714009AA34A94EFE03F9511
:1053600008A0EFF0DF8D7DBF83A70193F9D7EFF0A1
:105370001F8DE1B7B3C7A5008D8B3307C50081E74B
:105380008D4763EDC700AA87637EE50894218507F2
:105390008505A38FD7FEE3EBE7FE82809376350089
:1053A000AA8789CA942185078505A38FD7FE93F61E
:1053B0003700C5BF9376C7FF138606FE63F0C706A6
:1053C00083A3050083A2450083AF850003AFC5001A
:1053D00083AE050103AE450103A3850183A8C50182
:1053E0009385450223A0770003A8C5FF23A2570099
:1053F00023A4F70123A6E70123A8D70123AAC70105
:1054000023AC670023AE17019387470223AE07FF43
:1054100075B790419107910523AEC7FEE3EBD7FE28
:10542000E3E6E7F6828039713EDA2ED232D436D600
:105430003AD842DC46DE9387818122CC804326CA5B
:1054400006CEAA8409C41C4C99E32285352B0C4452
:1054500054102686228536C6EF007017F24062444B
:10546000D24421618280011126CA4AC806CE22CCCC
:105470004EC652C4AA842E8901C51C4D91E329232E
:105480009C4C804499E3268501239717000093875D
:10549000A743631BF402C0405E24A18BB1C71C4824
:1054A000A1C7FD59294A1C4483450900FD17B1E9EC
:1054B0001CC463DD07062286A9452685E120FD5729
:1054C0006308F502294535A0971700009387C74167
:1054D0006314F4008044C9B7971700009387C73C52
:1054E000E31CF4FAC0444DBFA2852685912A55D904
:1054F0007D55F2406244D2444249B249224A056194
:1055000082801CC4050963D70700184C63CAE700F2
:10551000638845011C401387170018C08CA361B72E
:10552000228626858520E31035F9D9B71C401387DC
:10553000170018C0294798A371B793878181AA855E
:1055400088436FF05FF205C68547630BF602138749
:1055500015002E968346F7FF0505BA87A30FD5FEE3
:1055600081CE0507E318E6FE2300050011A0AE87F3
:10557000850703C7F7FF6DFF3385B7407D15828030
:10558000AE87DDB7011122CC26CA4AC806CE4EC668
:10559000AA842E89328401C51C4D91E3F526971704
:1055A0000000938767326317F406C0401C4C1CC48C
:1055B0005E24A18BC1C31C48B5CF1C480840937919
:1055C000F90F1379F90F1D8D5C486346F500A2852C
:1055D0002685692C25E51C440505FD171CC41C40C7
:1055E0001387170018C0238037015C486388A70021
:1055F0005E24858B81CBA9476316F900A285268599
:10560000B5240DEDF24062444A85D2444249B24984
:1056100005618280971700009387072D6314F400BB
:10562000804469B79717000093870728E310F4F8C0
:10563000C044ADBFA2852685212041D17D59D9B76F
:1056400041119387818126C2844322C44AC006C681
:105650002A892E8489C49C4C99E326853526971780
:10566000000093876726631BF402C0400317C40041
:1056700093170701C18393F68700ADEA93F60701FC
:1056800095EEA5472320F900136707045AA47D551A
:10569000B24022449244024941018280971700009F
:1056A000938787246314F4008044C9B797170000D8
:1056B0009387871FE31CF4FAC0444DBF918B9DC3B1
:1056C0004C5889C9930744046384F5004A85292B03
:1056D000232A04025E242322040093F7B7FD5EA46C
:1056E0001C481CC05E2493E787005EA41C4899EB0D
:1056F0005E241307002093F707286385E700A2853F
:105700004A8591295E2413F717001DC35C482324A2
:105710000400B307F0401CCC1C480145B5FB8317BF
:10572000C40013F707082DD793E707045EA485B7D5
:10573000898B014791E3584818C4F9BFDE25011150
:1057400022CC26CA06CE4AC84EC613F78700AA84C2
:105750002E8479EBD841634DE000B841634AE00004
:105760000145F2406244D2444249B2490561828017
:1057700058547DD703A904009396370123A0040051
:1057800063DB060670485E24918B99C75C401D8ED2
:105790005C5899C33C401D8E5C540C508146268554
:1057A0008297FD575A24631DF5009440F54763E83E
:1057B000D706B70740208507B3D7D700858BA5C389
:1057C0001C48232204001CC09317370163D807002C
:1057D000FD576314F5009C4091E368C84C5823A022
:1057E0002401BDDD930744046384F5002685ED2E76
:1057F000232A0402B5B70C50014685462685029738
:10580000FD572A86E311F5F89C40B5DF754763859F
:10581000E70059476393E70423A0240191B7136776
:1058200007045AA47D5535BF83A90501E38A09F20F
:1058300003A905008D8B23A03501330939410147A8
:1058400091E3D84918C4E35D20F11C540C50CA867A
:105850004E86268582976347A0005E2493E707045F
:105860005EA4C9B7AA993309A940F1BF9C49A5C351
:10587000011122CC06CE2A8411C51C4D81E72EC60B
:105880002122B2459717000093870704639CF50017
:105890004C408397C5009DC722856244F240056154
:1058A0006FF0DFE997170000938707046394F50012
:1058B0000C44C5B797170000938707FFE39BF5FCDF
:1058C0004C44C1BFF24062440145056182800145FC
:1058D0008280411122C406C62A844EA572A52320C7
:1058E0000500232205002324050023220506232882
:1058F0000500232A0500232C0500214681451305B8
:10590000C505EFA05FC497170000938707B35CD06D
:1059100097170000938727B51CD49717000093872B
:1059200007B95CD497170000938767BB00D01CD8D9
:10593000B24022444101828097050000938545F3DF
:1059400091AA411126C2130680069384F5FFB38401
:10595000C4024AC02E8922C406C6938544070D2E70
:105960002A8401CD2320050023222501310508C406
:10597000138684068145EFA01FBD2285B2402244D4
:1059800092440249410182801C4DA5E7411106C69F
:1059900022C497070000938767FA1CD5938701827A
:1059A0009C432324050423260504232805046314AB
:1059B000F50085471CCD2A84352848C022851D283E
:1059C00008C42285052848C4484001469145EFF0A7
:1059D0005FF008440546A545EFF0BFEF484409468F
:1059E000C945EFF01FEF85471CCCB240224441016E
:1059F0008280828041119387018226C284434AC0FB
:105A000006C69C4C22C42A8981E72685EFF0DFF781
:105A1000938484048044DC40FD1763D607009C40D7
:105A2000B9CF8440C5BF0317C40039E7C1778507E4
:105A3000232204062320040023220400232404003C
:105A40005CC423280400232A0400232C04002146DC
:105A500081451305C405EFA01FAF232A0402232CA0
:105A6000040223240404232604042285B240224491
:105A700092440249410182801304840671BF91451A
:105A80004A85EFF01FEC88C049FDB1472320F9009B
:105A90000144E1BF797122D44AD052CC56CA5AC8C7
:105AA0005EC606D626D24ECE2A8AAE8A1304850456
:105AB0000149054BFD5B09ECB25022544A859254D2
:105AC0000259F249624AD24A424BB24B4561828046
:105AD000044483294400FD1963D409000040E1BF58
:105AE000DE24637BFB008397E40063877701A68550
:105AF0005285829A3369A90093848406E9BF19719B
:105B0000A6DAAE848395E500A2DC86DE328463DB10
:105B10000500DE2423A0060093F7070885E7930716
:105B200000401DA0300836C6EF00F021B246E34227
:105B300005FE7247BD67F98F7977BA9793B717005B
:105B40009CC2F1BF930700041CC0F6506654D654A3
:105B5000014509618280DE25011122CC06CE26CACC
:105B60004AC8898B2E8489CF930774041CC01CC833
:105B700085475CC8F2406244D24442490561828054
:105B800074003000AA84EFF09FF7A2452A89268589
:105B9000012219E98317C40013F7072061FFF19B65
:105BA00093E727005EA4C9B797070000938707D93A
:105BB0009CD45E2408C008C893E707085EA4A247E7
:105BC0005CC8B24781CF8315E4002685EF00D01A68
:105BD00011C55E24F19B93E717005EA45E24336930
:105BE000F9002316240179B7DDC183A7C5FF411150
:105BF00022C406C626C21384C5FF63D307003E94A1
:105C0000AA84EF00301F938781939C4381EF232266
:105C1000040023AC81922244B24026859244410183
:105C20006F00701D637EF40014403307D400639648
:105C3000E7009843DC43369718C05CC0D9BFBA87E9
:105C4000D84319C3E37DE4FE94433386D700631F32
:105C500086001040B29694C33386D700E31DC7FA7E
:105C600010435843B29694C3D8C375B76375C40044
:105C7000B1479CC04DB71040B306C4006316D700AF
:105C800014435843B29614C058C0C0C369B7828049
:105C9000011126CA93843500F19806CE22CC4AC859
:105CA0004EC6A104B14763F3F404B14463E2B40403
:105CB0002A89EF0030149387819398433A8439E01E
:105CC0009387C1939C4391E781454A85252F23AE55
:105CD000A192A6854A853D27FD5963193507B1472D
:105CE0002320F9004A85EF00101129A0E3D004FC1D
:105CF000B1471CC10145F2406244D2444249B24915
:105D0000056182801C40858F63CF0702AD4663F634
:105D1000F6001CC03E9404C031A05C4063138702AF
:105D200023ACF1924A85EF00100D1305B4009307E0
:105D3000440061993307F5405DDF3A94898F1CC0B8
:105D40005DBF5CC3C5B72287404095BF13043500D3
:105D50007198E30285FCB305A4404A856525E31CE0
:105D600035FBB5BF1C46FD171CC663DA0700184E8D
:105D700063C5E700A9476394F5006FF0BF801C423C
:105D80002E851387170018C28CA38280011122CCA4
:105D900026CA4AC84EC652C406CE2A89AE89328463
:105DA000B304D6007D5A63149400014509A80C2061
:105DB0004E864A85EFF01FFB0504E31645FFF240CF
:105DC0006244D2444249B249224A05618280357117
:105DD00022CD26CB4AC94EC706CF52C556C35AC19B
:105DE000DEDEE2DCE6DAAA89AE843289368409C5D1
:105DF0001C4D99E3EFF05FB9971700009387C7AC8C
:105E00006398F40C83A44900DE24A18BE5C79C4869
:105E1000F5C393070002A304F1029307000302D223
:105E20002305F10222C6930B5002971A0000938AB1
:105E3000AAAD054C294B4A841C2099C3639F770D5A
:105E4000B30C2441638E0C00E6864A86A6854E85F7
:105E5000EFF0DFF3FD57630FF51C9256E69636D24E
:105E60001C206389071CFD571309140002C802CEC9
:105E70003ECA02CCA309010482D483450900154619
:105E80005685A92F13041900C24751E913F70701DA
:105E900009C713070002A309E10413F7870009C724
:105EA0001307B002A309E104834609001307A00207
:105EB000638FE606F2474A848146254618209305FB
:105EC0001400130707FD6377E60AB5CA3ECE85A81E
:105ED00097170000938747A16395F40083A4890076
:105EE00025B7971700009387279CE39FF4F083A4BE
:105EF000C90019BFA6854E85EFF08FF419D97D55DD
:105F0000FA406A44DA444A49BA492A4A9A4A0A4B48
:105F1000F65B665CD65C0D618280050431BF33059B
:105F200055413315AC00C98F3EC82289B9B73247F5
:105F300093064700184336C6634707023ACE182037
:105F40009307E002631DF70418309307A002631B58
:105F5000F702B2470904138747009C433AC663C15E
:105F600007023ECA2DA83307E04093E727003ACE48
:105F70003EC8F1B7B387670385462E84BA973DBF05
:105F8000FD57C5B7050402CA81468147254618203A
:105F900093051400130707FD6374E606F9F20C205D
:105FA0000D46171500001305A5960D2D11CD971759
:105FB00000009387E7951D8D93070004B397A70012
:105FC000424505045D8D2AC80C20194617150000AE
:105FD00013054594130914002304B102012535C1AA
:105FE00097A7FFFF9387070295E74247B2471377CA
:105FF000071009CF91073EC69257D2973ED225BDD2
:10600000B387670385462E84BA9751B79D07E19BF6
:10601000A107D5B7780097060000938666D7268635
:106020000C084E8597000000E7000000FD572A8A03
:10603000E314F5FCDE2493F70704E39207EC125512
:10604000C1B5780097060000938686D426860C0892
:106050004E85012AE1BF797156CA9C49BA8A984592
:1060600022D426D24ECE52CC06D64AD05AC85EC6CC
:10607000AA892E84B284368A63D3E700BA879CC08B
:106080000347340419C385079CC01C4093F70702DB
:1060900081C79C4089079CC00329040013796900CB
:1060A000631A0900130B9401FD5B5C449840998FBF
:1060B000634CF9041C408346340493F70702B3365B
:1060C000D000A5EB13063404D2854E85829AFD5785
:1060D0006303F5041C4011469840998B5444814455
:1060E0006397C700B384E64063D3040081441C4433
:1060F00018486354F700998FBE94014969047D5B89
:1061000063982405014509A885465A86D2854E859F
:10611000829A631E75017D55B250225492540259E1
:10612000F249624AD24A424BB24B4561828005092C
:10613000ADBF3307D40013060003A301C704034710
:10614000540493871600A2978906A381E7049DBF94
:1061500085462286D2854E85829AE30E65FB050927
:1061600045B7797122D426D24AD04ECE06D652CC2B
:1061700056CA5AC8B689942D930790063289AA84C4
:106180002E8413863504638DF60263E2D7069307E7
:1061900080056386F61863EDD700638E06209307AB
:1061A0003004638EF60A930A24042301D404C9A0A0
:1061B000930730066385F60A93074006E395F6FEDB
:1061C0001C40084393F6070893054500C5C61C41CB
:1061D0000CC363D807001307D002B307F040A30134
:1061E000E4049706000093866673294765A8930721
:1061F00000076382F61663E5D7029307E00663891A
:10620000F6189307F006E390F6FA0C401C4313F8D7
:106210000508138547006307080608C39C4385A843
:1062200093075007E383F6FE930780076389F6120E
:1062300093073007E399F6F61C43D04181459386D6
:10624000470014C383AA07005685492E01C53305AC
:10625000554148C05C401CC8A301040461A81C430C
:10626000930A2404938647009C4314C32301F40437
:106270008547D5B793F607041C410CC3B9DAC207AA
:10628000C18781BF93F5050408C3C9D99E231307AD
:10629000F0066387E60E9706000093862668294776
:1062A000A30104044C400CC463C5050008406D996B
:1062B00008C099E3B28A89CDB28AB3F5E702FD1A24
:1062C000B6958C212380BA00B3D5E70263F0E70CC2
:1062D000A147631EF7001C40858B91CB58401C489A
:1062E00063C7E70093070003A38FFAFEFD1A330686
:1062F000564110C84E87CA867000A2852685EFF0E9
:106300009FD57D5A631D450B7D55B2502254925442
:106310000259F249624AD24A424B45618280A382C5
:10632000D504970600009386665F0C40084313F877
:1063300005081C411105630D080208C313F7150079
:1063400001C793E505020CC04147B9FB0C4093F52A
:10635000F5FD0CC0B1B79C4193E707029CC19307C0
:106360008007A302F404970600009386665C75BF5D
:1063700013F8050408C3E30308FCC207C1837DBF0B
:106380009706000093868659214719BFAE8735B717
:1063900094411C43CC4913F8060813854700630653
:1063A000080008C39C438CC339A008C393F60604B5
:1063B0009C43F5DA8EA323280400B28A25BF144833
:1063C0005686CA8526858299E30045F51C40898B4F
:1063D0008DE7B2474844E35AF5F23E853DB785461E
:1063E0005686CA8526858299E30065F3050A5C44D2
:1063F0003247998FE345FAFEE9BF014A930A9401B7
:106400007D5BF5B7411122C42A842E8597170020A1
:1064100023A4079C06C6EFC0FFB2FD576319F50021
:10642000971700209387479B9C4391C31CC0B240A1
:10643000224441018280411122C42E848395E500CB
:1064400006C65D2A634905007C48AA977CC8B2400D
:106450002244410182805E247D777D17F98F5EA4FE
:10646000FDB7DE25011122CC26CA4AC84EC606CE8B
:1064700093F70710AA842E843289B68991C7839531
:10648000E500894601460D225E247D777D17F98F50
:106490005EA48315E4006244F240CE864A86B24987
:1064A00042492685D244056125A8411122C42E8483
:1064B0008395E50006C6CD28FD575A24631AF500DA
:1064C000FD77FD17F98F5EA4B2402244410182801E
:1064D0008567D98F5EA468C8C5BF8395E50025A8E8
:1064E000411122C42A842E85B28536869717002052
:1064F00023A4078E06C6EFC01FA1FD576319F50040
:10650000971700209387478D9C4391C31CC0B240CE
:10651000224441018280411122C42A842E8597178A
:10652000002023AB078A06C61122FD576319F50028
:10653000971700209387478A9C4391C31CC0B240A1
:10654000224441018280411122C42A842E85B285D1
:106550009717002023A2078806C6CD20FD57631990
:10656000F50097170020938727879C4391C31CC091
:10657000B240224441018280411122C42A842E85E6
:106580009717002023AA078406C6C920FD57631960
:10659000F50097170020938727849C4391C31CC064
:1065A000B240224441018280411122C42A842E85B6
:1065B000B28536869717002023A0078206C6792861
:1065C000FD576319F500971700209387E7809C43D8
:1065D00091C31CC0B24022444101828093F5F50F63
:1065E0002A966314C500014582801C21E38EB7FE04
:1065F0000505C5BF82808280411122C42A842E8570
:10660000B28536869707002023A8077C06C6B928DE
:10661000FD576319F500970700209387E77B9C439C
:1066200091C31CC0B240224441018280930780057F
:10663000170700202322F77A7D5582809307800573
:1066400017070020232AF7787D558280930780055D
:10665000170700202322F7780145828093078005E1
:1066600017070020232AF7767D558280930780053F
:10667000170700202322F7767D55828053797374A3
:10668000656D436C6B3A25640D0A000043686970C0
:1066900049443A253038780D0A0000005631302E32
:1066A000342E36004672656552544F53204B657246
:1066B0006E656C2056657273696F6E3A25730D0AAC
:1066C0000000000073686F756C646E27742072752B
:1066D0006E20617420686572652121002E2E2F4680
:1066E00072656552544F532F706F727461626C659E
:1066F0002F4D656D4D616E672F686561705F342E3B
:1067000063000000657272206174206C696E652000
:106710002564206F662066696C6520222573222E11
:10672000200D0A20000000002E2E2F4672656552B3
:10673000544F532F706F727461626C652F474343DF
:106740002F524953432D562F706F72742E630000E1
:106750002E2E2F4672656552544F532F71756575F5
:10676000652E63002E2E2F4672656552544F532FAF
:106770007461736B732E630049444C450000000044
:10678000002D0000002D0000402D00004C2D0000C9
:106790008E2D0000002D0000002D0000402D000077
:1067A0004C2D0000546D7251000000002E2E2F461B
:1067B00072656552544F532F74696D6572732E6301
:1067C00000000000546D722053766300636F6D6D9E
:1067D0006F6E5461736B00007472616E736D6974D7
:1067E0005461736B000000005570526563656976F3
:1067F000655461736B000000446F776E526563658A
:106800006976655461736B005B494E464F5D205B52
:1068100025733A25645D2073656E64204A355F30C8
:106820002044617461203A202573202C2025640ABD
:106830000D0A00005B494E464F5D205B25733A25EB
:10684000645D20696E2047575F4D736750726F63B8
:1068500046756E635F446973747269627574696FBB
:106860006E5F50726F66696C650A0D0A0000000069
:106870005B494E464F5D205B25733A25645D206978
:106880006E2047575F4D736750726F6346756E6336
:106890005F526561645F50726F66696C650A0D0ACC
:1068A00000000000000000000000000000000000E8
:1068B00000000000000000000000000000000000D8
:1068C00000000000000000000000000000000000C8
:1068D00000000000000000000000000000000000B8
:1068E00000000000000000000000000000000000A8
:1068F0000000000000000000000000000000000098
:1069000000000000232D302B20000000686C4C009C
:1069100065666745464700003031323334353637D7
:10692000383941424344454600000000303132339B
:1069300034353637383961626364656600000000BB
:10694000000000000000000001020304060708091F
:106950000000000001020304010203040607080905
:10696000000000000600000080250000000000007C
:106970000000000000000000000000000000000017
:10698000000000000000000007000000802500005B
:1069900000000000000000000000000000000000F7
:1069A00000000000000000000000000002000000E5
:1069B0008025000000000000000000000000000032
:1069C00000000000000000000000000000000000C7
:1069D000080000008025000000000000000000000A
:1069E00000000000000000000000000000000000A7
:1069F00000000000030000008025000000000000EF
:106A00000000000000000000000000000000000086
:106A100000000000000000000500000000C20100AE
:106A20000000000000000000000000000000000066
:106A3000000000000000000000000000624A0000AA
:106A4000010000008A4B000002000000864B00009D
:106A500003000000D64A000004000000C84A0000FD
:106A600005000000BA4A000006000000AC4A000021
:106A7000070000009E4A000008000000904A000045
:106A800009000000824A00000A000000744A000069
:106A90000B000000664A000003000000744B000079
:106AA00004000000624B000005000000504B000095
:106AB000060000003E4B0000070000002C4B0000C9
:106AC000080000001A4B000009000000084B0000FD
:106AD0000A000000F64A00000B000000E44A000033
:106AE00000000000C4680000E4680000A468000022
:106AF0000000000000000000000000000000000096
:106B00000000000000000000000000000000000085
:106B10000000000000000000000000000000000075
:106B20000000000000000000000000000000000065
:106B30000000000000000000000000000000000055
:106B4000006CDC0202040608AAAAAAAA040000003B
:106B5000D86D002001000000A0010020008000206E
:086B6000A0010020000000006C
:00000001FF
